:1039EC000F580F4E0F430F380F2D0F210F140F07C9
:1039FC000EF90EEB0EDC0ECC0EBC0EAB0E9A0E8737
:103A0C000E750E610E4D0E380E220E0C0DF40DDCE3
:103A1C000DC40DAA0D900D750D5A0D3E0D210D0303
:103A2C000CE40CC50CA50C850C640C420C200BFD95
:103A3C000BD90BB50B900B6B0B460B200AF90AD369
:103A4C000AAC0A840A5D0A350A0D09E409BC09931B
:103A5C00096B0942091A08F108C808A0087808502F
:103A6C000828080007D807B1078A0764073E07181B
:103A7C0006F206CD06A906840661063E061B05F86D
:103A8C0005D705B50595057405550535051704F9D4
:103A9C0004DB04BE04A20486046A044F0435041B30
:103AAC00040203E903D103B903A2038B0375035F7B
:103ABC00034A03350321030D02FA02E702D502C3C0
:103ACC0002B102A0028F027F026F025F025002411C
:103ADC00023302250217020A01FD01F001E301D7AE
:103AEC0001CC01C001B501AA019F0195018B018197
:103AFC000178016E0165015C0154014B0143013BEE
:103B0C000133012C0125011D0116011001090102CF
:103B1C0000FC00F600F000EA00E500DF00DA00D45B
:103B2C0000CF00CA00C600C100BC00B800B300AF93
:103B3C0000AB00A700A3009F009B0098009400918D
:103B4C00008D008A00870084008100010C010105B2
:103B5C0002011E030A9604013205030306006407E2
:103B6C00010108000009015A0E01010F00011200A9
:103B7C006413010114013C1501FA1664FA17FFFFD6
:103B8C001D00072000072400022701012F013C30F3
:103B9C00020232010335FFFF3603073C00143DFFE0
:103BAC00FF180002191E461A00021B00022D32C813
:063BBC002E0001FAFAFAE6
:10004800900785E0FEA3E0FF7457BE0010D39F40E1
:100058000C903B5612001EE493F599801290078588
:10006800E0FEA3E0FF903B5612001EE493F5999042
:10007800078512000E900785E0FEA3E0FF746C6F01
:100088004E700375130022900071E0B402087401E9
:10009800900071F0D20C900139E0900029F09001A5
:1000A8003AE090002AF090013BE090002BF0A20A81
:1000B800B34016900139E0700C90013AE070069058
:1000C800013BE060028002C20A900139E0B4300FBF
:1000D80090013AE0B4470890013BE0643B6002803D
:1000E80004D20B8002C20BE558B40102800302025D
:1000F80011900056E0F566900061E0F568900062A6
:10010800E0F569900073E0F56A900079E0900028C6
:10011800F090007BE0F56590007CE0F56790007F4B
:10012800E0F564900080E0F56390008FE090004077
:10013800F0900090E0900041F0900091E090004233
:10014800F0900092E0900043F0900093E09000441B
:10015800F0900094E0900045F0900095E090004603
:10016800F0900096E0900047F0900098E090003200
:10017800F0900099E0900033F090009AE0900034FD
:10018800F090009BE0900035F0900078E0B4011703
:1001980090000A740FF0A374FFF090000CE4F0A331
:1001A800F07402900078F0900078E0B40359900061
:1001B8000CE0FEA3E0FF90000AE0FCA3E0FD1200C3
:1001C800037410123D227408123D14EF900025F0BC
:1001D800EF700674FF900025F07400900078F0909E
:1001E800000BE0900026F090000AE0900027F090C5
:1001F8000025E0900788F0900026E0900789F090AD
:100208000027E090078AF0803F900080E070067534
:100218005801756300A20AB3402E900139E090009E
:1002280029F090013AE090002AF090013BE090001C
:100238002BF0900029E0700C90002AE070069000E6
:100248002BE060028002C20AE5667003756602E56B
:100258006870037568027E847FBCE5668E048F052E
:10026800FF123D048C398D3AE56975F0FAA4FFAEAA
:10027800F0E5688E048F05FF123D048C3D8D3E909D
:10028800004EE0F56090004CE0FE900068E0B50696
:100298001890004BE0FE900067E0B5060C90004A0D
:1002A800E0FE900058E06E606F900068E070069085
:1002B8000067E060067400900058F0900068E0B4B1
:1002C80002089000487401F08005900048E4F0901E
:1002D8000067E0B402089000497401F080059000BE
:1002E80049E4F0900067E06006900049E060028011
:1002F800057560048003756005E559B55802D20C90
:10030800900067E090004BF0900068E090004CF09F
:10031800900058E090004AF022E5B554F7F5B5E5AD
:10032800B554FDF5B5C287C290C292756F00E5B5A8
:1003380054DFF5B5C207E5B554FBF5B5755105E5CC
:100348005104F55290004EE0F560C211C212C2137A
:10035800C209E5B554FEF5B5C28E758D00758B00E2
:10036800754C00752600752500D28E22750A007519
:100378000900AE09AF0A7457BE00039F5003020478
:1003880031903B5612001EE49390004D123D3A0FF7
:10039800BF00010EE0FC903B5612001EECFEE493F9
:1003A800FFEEC39F5026AE09AF0A0FBF00010E90A3
:1003B8003B5612001EAE09AF0AE493FC903B56125E
:1003C800001EE49390004D123D3AECF0AE09AF0ADE
:1003D800903B5612001EE49390004D123D3AE0FC0B
:1003E800903B5812001EECFCE493FDECD39D4019A1
:1003F800903B5812001EE493FC903B5612001EE4FA
:100408009390004D123D3AECF0AE09AF0A74022FFA
:10041800FF50010E8E098F0A780A740126F65004DF
:1004280018E436F6400302037A22750A00750900BB
:10043800AE09AF0A7415BE00039F50030204FF9073
:100448003BAD12001EE49390004D123D3A0FBF00E1
:10045800010EE0FC903BAD12001EECFEE493FFEEB3
:10046800C39F5026AE09AF0A0FBF00010E903BADE7
:1004780012001EAE09AF0AE493FC903BAD12001EB9
:10048800E49390004D123D3AECF0AE09AF0A903B70
:10049800AD12001EE49390004D123D3AE0FC903BF3
:1004A800AF12001EECFCE493FDECD39D4019903B89
:1004B800AF12001EE493FC903BAD12001EE4939033
:1004C800004D123D3AECF0AE09AF0A740F6F4E7052
:1004D80006750A15750900AE09AF0A74022FFF5098
:1004E800010E8E098F0A780A740126F6500418E462
:1004F80036F6400302043822054D22054C22054EEB
:10050800C2CF2290F800E4936406600280FE7584EE
:100518000175A70075FF80900787E4F075C910750D
:10052800A70F75A1C775A70075D90075CEFF75A768
:100538000F75F1FE75F2FF75F33775F47875A4BA87
:1005480075A5FF75A60775AE0075AFFF75D48175E3
:10055800D5FF75D6FF75D7FFC293C294C291C287E3
:10056800C290C292C2A1E5B554BFF5B5E5B554DF56
:10057800F5B5E5B554EFF5B5E5B5547FF5B5E5B591
:1005880054F7F5B5E5B554FDF5B575A70075A201A5
:1005980075A14775F80975BC0175BE0475BD6C7504
:1005A800BE0775BDA075BE0875BD0175BC0075BBDD
:1005B8001875BC2075BA0875E88075D11375A70F32
:1005C80075E10575E20075C74075970075978074E9
:1005D8000A123CF47597C0E5975420700280F875AC
:1005E8008F0275A700D2AF75980075A90C75A70F73
:1005F80075AB4375ADFB75AC1E75A7007589117594
:100608008E00758C00758A00D2A9D28C758D007504
:100618008B00D2ABD28E75CD0075CC0075CA007533
:10062800CB00D2ADC2CFD2CA759104759200759332
:10063800CD75EF0675D94075CF01900785E4F0A315
:10064800F0751300751400C299D20AC2141203215E
:1006580074C8F51875170012231B75A70FE5FB90D2
:10066800001AF0E5FA90001BF0E5F990001CF0750F
:10067800A70090F800E493F50812245212298C90F0
:100688000788E0900025F0900789E0900026F09018
:10069800078AE0900027F090078BE0900028F09000
:1006A800078CE0F56690078DE0F56890078EE0F519
:1006B8006990078FE0F56A900790E0F565900791DB
:1006C800E0F567900792E0F564900793E0F5639092
:1006D8000794E0900029F0900795E090002AF090A8
:1006E8000796E090002BF0900797E0900040F0907C
:1006F8000798E0900041F0900799E0900042F09050
:10070800079AE0900043F090079BE0900044F09037
:10071800079CE0900045F090079DE0900046F0901F
:10072800079EE0900047F090079FE0900032F0901D
:1007380007A0E0900033F09007A1E0900034F0901B
:1007480007A2E0900035F07400900081F090013924
:10075800E0700C90013AE0700690013BE060028086
:1007680004C20A8002D20A90F807E493900021F0AC
:10077800900021E0440A900021F0900021E054FE0E
:10078800900021F07406900012F07402900013F0AB
:1007980090F802E493900014F07403900015F0743C
:1007A80003900016F07424900017F0740590001858
:1007B800F07405900019F090F804E49390001DF08F
:1007C800740090001EF090F805E49390001FF090DC
:1007D800F806E493900020F074FF900022F0744D26
:1007E800900124F07465900125F07472900126F050
:1007F8007463900127F07420900128F074379001F9
:1008080029F0743290012AF0743290012BF0742E82
:1008180090012CF0743690012DF0742090012EF088
:10082800743590012FF07453900130F0745090019A
:1008380031F07444900132F0900079E0D394014093
:10084800067400900079F075580175590174039089
:10085800004BF012008F12037412043212234775F2
:100868004C00E5B554FEF5B5C211C212C21390078B
:1008780085E4F0A3F0752400752300754800752AF7
:1008880000752900754900753200753100754A00F8
:10089800755400755500755A0075510575520175E6
:1008A800343C7533007571007570007572CD7556DE
:1008B800007557007543007544007545007546007E
:1008C800755B00754700754200754100900006E4AD
:1008D800F0A3F0900008E4F0A3F0755E00755F00E7
:1008E80090000E74FDF0A374E8F0900023E4F07417
:1008F80064900024F0C200D201C202D203754D00F8
:10090800756D00C295C296C2A0C297C2A2C20C7EE3
:10091800017F00900027E0123D22900026E02FFF83
:1009280050010E90000AEEF0A3EFF0900025E07061
:100938000674FF900025F090000AE0FEA3E0FFEFA8
:10094800D394FFEE940F400790000AE4F0A3F074EC
:1009580000900070F07400900078F07400900081AE
:10096800F0740090008CF074009000B3F0E56770AC
:1009780003756704743A90074DF074FD90074EF0C4
:10098800900413E0900453F0D2B0D2B7D2A7D2A605
:10099800D2B1D2A3C207A2B6B39204A2B3B392054E
:1009A800D29CD2EC75CF01A298B34005C298122C04
:1009B800F0E5136006A299B3B340028005C299120C
:1009C8003260E51464016005E514B4040280D5E5DD
:1009D8004DD39405400CE55AC394C85002055A7586
:1009E8004D00E572C394F0501A787012003FAE7053
:1009F800AF71EFD394E8EE94034008057275710067
:100A0800757000C28E7E047F00E54C123D22E58D94
:100A180075F004A4FDACF0EF2DFDEE3CFCE58B7504
:100A2800F04084FF7E00ED2FFFEC3EFE8E258F26E2
:100A3800D28EA2B6300401B35003020BADA2B63079
:100A48000401B35003020BADA2B65003020AE90534
:100A580054A214400575FFA0D214E5B54401F5B5BC
:100A6800900024E4F0E554D3956640737C847DBC03
:100A7800AE25AF26123BC28E238F24E5482FFF50A8
:100A8800010E7401123D148E238F24852448755459
:100A980001C28E758D00758B00754C00D28EE524D1
:100AA8004523600E7406BE0009D39F4005A211B30A
:100AB80040028005755A00D20EAE23AF247405BEDD
:100AC80000039F5005A211B34002800BD21175514B
:100AD80001755201755A0AE543B40603754300D2FD
:100AE80004A2B6B35003020BADC20490006AE060E2
:100AF800181233A1A200B34008E5B54408F5B58043
:100B080006E5B554F7F5B58002C20090006DE060C7
:100B1800181234F6A202B34008E5B54402F5B580D0
:100B280006E5B554FDF5B58006E5B554FDF5B5A265
:100B380007B34004D2A08002C2A0900058E060042D
:100B4800D2978002C297900049E0B40104D2958000
:100B580002C295900048E0B40104D2968002C29681
:100B6800A209B34004D2A28002C2A2900018E0FEFB
:100B7800900014E0C39E4009900014E0D39408400C
:100B88000974FB900023F012032190001DE060150A
:100B980090001DE0FE900017E06E600974FE900062
:100BA80023F0120321C2CA7E017F00E54E123D22C6
:100BB800E5CD2FFF50010E8E278F28D2CAE565B4E8
:100BC800014890000EE0FCA3E0FDEFC39DEE9C40C1
:100BD80039B208E52A45296013A208B34008E5B5EB
:100BE8004404F5B58006E5B554FBF5B590000EE074
:100BF800FEA3E0FF900010E0FCA3E0FDEF2DFDEE6A
:100C08003CFC90000EECF0A3EDF0A2B3300501B36C
:100C18005003020CFBA2B3300501B35003020CFBD6
:100C2800A2B35003020CF40555A214400575FFA0A9
:100C3800D214E5B54401F5B5900024E4F0E555D3A8
:100C480095685003020CF27CEA7D60AE27AF28124B
:100C58003BC28E298F2AE569123D2274FF8E048FCC
:100C680005FF123D048C298D2AE5492DFD50010C04
:100C780074018C068D07123D148E298F2A852A4906
:100C8800A209B340157464123D22900066E08E04F8
:100C98008F05FF123D048C298D2A75550190000E91
:100CA800E0FEA3E0FFAC27AD2812000390000EEE93
:100CB800F0A3EFF0E567FF123D04740AFF123D044C
:100CC80090007AE08C068D07123D2274148E048FF2
:100CD80005FF123D04900010ECF0A3EDF0C2CA75B8
:100CE800CD0075CC00754E00D2CAD205A2B3B34070
:100CF80002C205A211B3B35007E556C394064003D8
:100D0800021312E56D9022CDF8282873900058E060
:100D1800C394024003020E68E551D39401500302C4
:100D28000E68E55175F040A4FFAEF0900311120073
:100D38001EE0C395455018E55175F040A4FFAEF08C
:100D480090031012001EE0F52E752D00020E68E5C6
:100D58005175F040A4FFAEF090030F12001EE0C3DF
:100D680095454003020E04E55175F040A4FFAEF02E
:100D780090031012001EE55175F040A4FFAEF0E09C
:100D8800FC90030E12001EECFEE0FFEEC39FFEE592
:100D9800518E0475F040A4FFAEF090030F12001EB0
:100DA800E0F40425458C0088F0A4FFAEF0E5518FEF
:100DB800048E0575F040A4FFAEF090031112001EDA
:100DC800E55175F040A4FFAEF0E0FA90030F120071
:100DD8001EEAFEE0FFEEC39FFECDCCCD8E07123D8E
:100DE80004E55175F040A4FFAEF090030E12001E0A
:100DF800E02DFD50010C8C2D8D2E8064E55175F091
:100E080040A4FFAEF090030E12001EE55175F040AD
:100E1800A4FFAEF0E0FC90030D12001EECFEE0FF14
:100E2800EEC39F8545F0A4FFAEF0E5518F048E0513
:100E380075F040A4FFAEF090030F12001EE0FECD47
:100E4800CCCD8E07123D04E55175F040A4FFAEF0FD
:100E580090030D12001EE02DFD50010C8C2D8D2EDF
:100E6800756D01021312900058E0C394024003020A
:100E7800101C90004EE0D395515003020FC4E55169
:100E880075F040A4FFAEF090031712001EE0C39562
:100E9800455018E55175F040A4FFAEF090031612C6
:100EA800001EE0F52C752B00020FC4E55175F040CB
:100EB800A4FFAEF090031512001EE0C39545400351
:100EC800020F60E55175F040A4FFAEF090031612D2
:100ED800001EE55175F040A4FFAEF0E0FC9003144D
:100EE80012001EECFEE0FFEEC39FFEE5518E047576
:100EF800F040A4FFAEF090031512001EE0F40425A4
:100F0800458C0088F0A4FFAEF0E5518F048E05757E
:100F1800F040A4FFAEF090031712001EE55175F0E3
:100F280040A4FFAEF0E0FA90031512001EEAFEE0BE
:100F3800FFEEC39FFECDCCCD8E07123D04E5517563
:100F4800F040A4FFAEF090031412001EE02DFD50F7
:100F5800010C8C2B8D2C8064E55175F040A4FFAEFC
:100F6800F090031412001EE55175F040A4FFAEF096
:100F7800E0FC90031312001EECFEE0FFEEC39F8519
:100F880045F0A4FFAEF0E5518F048E0575F040A43E
:100F9800FFAEF090031512001EE0FECDCCCD8E07FB
:100FA800123D04E55175F040A4FFAEF09003131212
:100FB800001EE02DFD50010C8C2B8D2CE551B40149
:100FC80023E560D39401401CE55604D395514014A1
:100FD800E545C39405500D90035EE0A829B80006C6
:100FE800952A40028003755102E551B560229000B0
:100FF8004EE0D395514019E55175F040A4FFAEF08D
:1010080090031612001EE0A823B80006952440029B
:1010180080020560756D02021312900058E0B40258
:101028002AE55175F040A4FFAEF090031612001E99
:10103800E0F52C752B00E55175F040A4FFAEF0905B
:10104800030D12001EE0F52E752D00900058E0B437
:10105800030F900050E0F52C752B00752E00752DB0
:1010680000756D03021312E55175F040A4FFAEF050
:1010780090031F12001EE0C3955A400302114890C6
:101088000048E07036E551D394014029AE23AF24DF
:10109800AC2DAD2EEDD39FEC9E401AE55175F04076
:1010A800A4FFAEF090031D12001EE0A829B80005A9
:1010B800D3952A5002800215518034E551D3940209
:1010C8004029AE23AF24AC2DAD2EEDD39FEC9E402E
:1010D8001AE55175F040A4FFAEF090031D12001EF2
:1010E800E0A829B80005D3952A500280021551E5D9
:1010F80051B55237E551C395605030E55604D39544
:10110800514028AE23AF24AC2BAD2CEFD39DEE9CE1
:101118004019E55175F040A4FFAEF090031E12008F
:101128001EE0A829B80006952A400280020551E56C
:10113800B554DFF5B5E55165526005C207755A002B
:10114800756D04021312E55175F040A4FFAEF090DE
:10115800031912001EE0B40117E55175F040A4FF11
:10116800AEF090031F12001EE0240AC3955A4003F4
:1011780002121E753064752F00A207B3500B900041
:101188005FE02405C39545400302121EE55175F042
:1011980040A4FFAEF090031C12001EE0C39545402A
:1011A80064E55175F040A4FFAEF090031B12001ED9
:1011B800E55175F040A4FFAEF0E0FC90031A120070
:1011C8001EECFEE0FFEEC39F8545F0A4FFAEF0E500
:1011D800518F048E0575F040A4FFAEF090031C12E9
:1011E800001EE0FECDCCCD8E07123D04E55175F012
:1011F80040A4FFAEF090031A12001EE02DFD50012E
:101208000C8C2F8D30AE23AF24AC2FAD30EFD39D97
:10121800EE9C4002D207756D05021312E551B40128
:1012280009900058E0C3940240030212F290035759
:10123800E0D3954550030212F2900355E0C395455B
:101248005040900356E0FE900354E0F4042EFE90C4
:101258000355E0F40425458E0088F0A4FFAEF09015
:101268000357E0FC900355E0F4042C8E048F05FF2F
:10127800123D04900354E02DFD50010C8C2B8D2C55
:10128800802C900354E0FE900353E0F4042E85452F
:10129800F0A4FFAEF0900355E08E048F05FF123DD9
:1012A80004900353E02DFD50010C8C2B8D2CE5513F
:1012B800C395605030E55604D395514028AE23AF0E
:1012C80024AC2BAD2CEFD39DEE9C4019E55175F065
:1012D80040A4FFAEF090031E12001EE0A829B8003B
:1012E80006952A40028003755102900048E0B40137
:1012F80006E551640160028003755102E5516552AB
:0A1308006005C207755A00756D00FC
:1022CD00020D14020E6E02102202106F02114E0248
:0222DD001224C9
:1013120090004FE02402A823B80007D3952440028E
:10132200C207A211B3B35009900058E0C39403401E
:10133200030214C3900048E060030213FDE551D399
:1013420094014049E55175F040A4FFAEF090031FAF
:1013520012001EE0C3955A5034E55175F040A4FFC7
:10136200AEF090031312001EE0A823B8001FD3951D
:1013720024401AE55175F040A4FFAEF090031E120E
:10138200001EE0A829B80005D3952A500280021554
:1013920051E551D39401402FE55175F040A4FFAEC1
:1013A200F090031112001EE0C39545501AE55175E5
:1013B200F040A4FFAEF090031D12001EE0A829B871
:1013C2000005D3952A500280021551E551D39401AC
:1013D2004022E55604C39551501AE55175F040A4D8
:1013E200FFAEF090031D12001EE0A829B80005D33D
:1013F200952A5002800215510214B8E551D3940285
:101402004049E55175F040A4FFAEF090031F120071
:101412001EE0C3955A5034E55175F040A4FFAEF07A
:1014220090031312001EE0A823B8001FD395244096
:101432001AE55175F040A4FFAEF090031E12001E93
:10144200E0A829B80005D3952A500280021551E57B
:1014520051D39402402FE55175F040A4FFAEF090B5
:10146200031112001EE0C39545501AE55175F04074
:10147200A4FFAEF090031D12001EE0A829B80005DB
:10148200D3952A500280021551E551D3940240228D
:10149200E55604C39551501AE55175F040A4FFAECC
:1014A200F090031D12001EE0A829B80005D3952A6A
:1014B200500280021551E55165526005C207755A06
:1014C2000090005FE0D395455009900053E0C3952A
:1014D200455002C207900058E07003021728A2A5E7
:1014E200B34008A2A4B34003021711AE35AF36745D
:1014F20041D39F749C9E4005783512003FAE35AFB4
:1015020036EFB48806EEB4130280030216EEA2A5EB
:1015120050030215B1900058E0B4010B90004EE068
:10152200D3956040020560900058E0B40254E55142
:1015320075F040A4FFAEF090031F12001EE0C395A9
:101542005A503F90004EE0D395514021E55604D3C6
:1015520095514019E55175F040A4FFAEF090031388
:1015620012001EE0A823B80006952440028002055E
:101572005190004EE0F560E55165526005C2077575
:101582005A00900058E0B4032690004EE0D39551E3
:101592004008E55604D3955150028002055190004F
:1015A2004EE0F560E55165526005C207755A00A22A
:1015B200A450030216EE900058E0B4016E90004869
:1015C200E07035E551D394014029E55175F040A40E
:1015D200FFAEF090031D12001EE0A829B8000FD341
:1015E200952A400A1551755A00855160800385512C
:1015F2006080037560018033E551D394024029E590
:101602005175F040A4FFAEF090031D12001EE0A839
:1016120029B8000FD3952A400A1551755A008551F1
:101622006080038551608003756002900058E0D3AA
:10163200940150030216E2E55175F040A4FFAEF0AA
:1016420090031F12001EE0C3955A40030216E29057
:101652000048E07041E551D394014034E55175F002
:1016620040A4FFAEF090031012001EE0A823B800C1
:101672001FD39524401AE55175F040A4FFAEF090B7
:10168200031D12001EE0A829B80005D3952A5002B6
:1016920080021551803FE551D394024034E55175E3
:1016A200F040A4FFAEF090031012001EE0A823B891
:1016B200001FD39524401AE55175F040A4FFAEF007
:1016C20090031D12001EE0A829B80005D3952A50E8
:1016D2000280021551E55165526005C207755A0034
:1016E200E556B40704055E8003755E00E563B40148
:1016F2000EAE35AF36EF64407005EE649C6002803A
:101702000EA2A54003755801A2A44003755802A277
:10171200A5B3B35006A2A4B3B34002800675360047
:10172200753500021816A2A5B34008A2A4B340035F
:10173200021802AE35AF367441D39F749C9E4005A9
:10174200783512003FAE35AF36EFB48806EEB413EB
:10175200028003021802A2A5406F900067E0605A5F
:10176200900049E0B40107900049E4F0800690003F
:10177200497401F0900049E07005756004800375BA
:101782006005900049E0B40104D2958002C295E55B
:1017920051B4051AE55175F040A4FFAEF090031D57
:1017A20012001EE0A829B80005D3952A500280082D
:1017B200755104C207755A008003756005E556B479
:1017C2000704055E8003755E00A2A44033900068A2
:1017D200E06021900048E0B40107900048E4F08006
:1017E200069000487401F0900048E0B40104D296DB
:1017F2008002C296E556B40704055E8003755E005A
:10180200A2A5B3B35006A2A4B3B3400280067536B4
:1018120000753500E55865596006900081E0600367
:1018220002199EC29C751400751300C2CAE5589035
:1018320022DFF8282873801212298C800D122A6563
:0A1842008008122B3E8003122C17C1
:0F22DF0002183802183A02183F02184402184930
:10184C00900028E0900079F0E566900056F0E5688D
:10185C00900061F0E569900062F0E56A900073F029
:10186C00E56590007BF0E56790007CF0E564900006
:10187C007FF0E563900080F0900029E0900139F052
:10188C0090002AE090013AF090002BE090013BF0A0
:10189C00900040E090008FF0900041E0900090F0BC
:1018AC00900042E0900091F0900043E0900092F0A4
:1018BC00900044E0900093F0900045E0900094F08C
:1018CC00900046E0900095F0900047E0900096F074
:1018DC00900032E0900098F0900033E0900099F086
:1018EC00900034E090009AF0900035E090009BF06E
:1018FC007400900081F0744D900124F07465900197
:10190C0025F07472900126F07463900127F0742016
:10191C00900128F07437900129F0743290012AF06C
:10192C00743290012BF0742E90012CF074369001CF
:10193C002DF0742090012EF0743590012FF074531B
:10194C00900130F07450900131F07444900132F0F9
:10195C00900413E0900453F0743A90074DF074FD2A
:10196C0090074EF012008F900004E4F0A3F090006A
:10197C00067475F0A37430F09000087475F0A374BD
:10198C0030F0855859D2CA754C00D29C741B90000B
:10199C0023F0E55165526006A211B3B34002806199
:1019AC00C207E5519022EEF82828738036D20E80BB
:1019BC0032E552B40102D20EE552B40302D20F80CA
:1019CC0022E552B40202D20FE552B40402D21080C6
:1019DC0012E552B40302D210E552B40502D20E80C5
:0319EC0002D20E16
:1022EE000219B70219B90219BD0219CD0219DD0280
:0222FE0019EDD8
:1019EF00AE29AF2A7405BE00039F5007E545D39477
:1019FF000550028006E5B54420F5B585515290009B
:101A0F0089E0D3955A500DC20EC20FC210E556B4DD
:101A1F000802D210E595C394EE400FC293C294C250
:101A2F0091E556B40802D2108015A20EB34002D22F
:101A3F0093A20FB34002D294A210B34002D291905E
:101A4F000071E06058E54575F00284FF7E0090015B
:101A5F004D12001EE0F55CE54775F00A84FF7E002D
:101A6F0090024D12001EE0F55DE55C255DD3946498
:101A7F00400BE55C255DC39464F55C8003755C00E9
:101A8F00E55C75F00284FF7E008F5CEFC3943350EA
:101A9F0007EF24CDF55C8003755CFF801CE5457571
:101AAF00F00284FF7E0090014D12001EE075F002DF
:101ABF0084FF7E00EF24CDF55CE54575F00284FFD1
:101ACF007E0090017F12001EE075F00284FF7E0001
:101ADF00EF24CDF56FE556902300F8282873806A20
:101AEF008068806680648062AE23AF247405BE0078
:101AFF00039F5005A212B34002800DD212755101FF
:101B0F00755202755A00D20E8040755CE1756FDD1B
:101B1F008038756FCDAE23AF247405BE00039F5080
:101B2F0005A212B34002800DD212755101755202F7
:101B3F00755A00D20E8013A211B34008755CE1757F
:0A1B4F006FDD8006755CCD756FCD6B
:10230000021AED021AEF021AF1021AF3021AF5028A
:0B2310001AF7021B19021B21021B46DA
:101B5900E595C3955C4004C2878002D287E556C3E8
:101B69009406500FA20EB3500AA20FB35005A2104B
:101B7900B340028003756FCDE595C3956F5004D2CC
:101B8900928002C292A207B34005E556B4070375D5
:101B990072CDE595C395724004C2908002D290E55A
:101BA90043C394064003022190A2EDB350030221DE
:101BB90090C2EDE5436003021D0D7E017F00E5BE85
:101BC900123D22E5BD2FFF50010E900000EEF0A35B
:101BD900EFF0900028E0B401177E0F7FFF9000001E
:101BE900E0FCA3E0FD120003900000EEF0A3EFF08B
:101BF900900078E0B4025B900000E0FEA3E0FF9063
:101C0900000AE0FCA3E0FDEDD39FEC9E400F90009D
:101C190000E0F8A3E090000AC8F0A3C8F090000023
:101C2900E0FEA3E0FF90000CE0FCA3E0FDEFD39DF4
:101C3900EE9C400F900000E0F8A3E090000CC8F083
:101C4900A3C8F0900000E0FEA3E0FF7404123D1465
:101C59008F44900078E07060900000E0FEA3E0FF00
:101C690090000AE0FCA3E0FDEFD39DEE9C400D122D
:101C79000003900000EEF0A3EFF08007900000E46D
:101C8900F0A3F0900000E0FEA3E0FF7410123D22E3
:101C9900900025E08E048F05FF123D04900000ECB2
:101CA900F0A3EDF07400D39D74019C4008900001ED
:101CB900E0F54480037544FFE54475F00AA4FFAEDE
:101CC900F074198E048F05FF123D048D45ED253200
:101CD900FFAE3150010E7401123D148F4585453216
:101CE900753100EFD394624003754562900071E04D
:101CF90064016006900065E060028005754301801B
:101D09000375BB17E543B401028003021DC87E01B8
:101D19007F00E5BE123D22E5BD2FFF50010E900068
:101D290000EEF0A3EFF0900071E0B4017CE53445DA
:101D3900336025AC33AD341DBDFF011C8F028E030A
:101D49008C068D079039EC12002EE493FE740193F2
:101D5900FFEFC39AEE9B400280057833123D4CAEEB
:101D690033AF3474B3BE0025D39F4021900000E007
:101D7900FCA3E0FD0FBF00010E9039EC12002EE428
:101D890093FE740193FFEDC39FEC9E40028005789A
:101D99003312003FAE33AF34E56A123D2274648ECC
:101DA900048F05FF123D048D47900071E0640260C5
:101DB90006900065E0600575BB168003754302E572
:101DC90043B402028003021EB67E017F00E5BE1203
:101DD9003D22E5BD2FFF50010E900000EEF0A3EF6C
:101DE900F0900071E0B4027EE53445336025AC33F0
:101DF900AD341DBDFF011C8F028E038C068D07902B
:101E0900388212002EE493FE740193FFEFC39AEE19
:101E19009B400280057833123D4CAE33AF3474B326
:101E2900BE0025D39F4021900000E0FCA3E0FD0FF8
:101E3900BF00010E90388212002EE493FE740193C4
:101E4900FFEDC39FEC9E40028005783312003FAE40
:101E590033AF34E56A123D2274648E048F05FF1294
:101E69003D048D478033900065E0602D900000E0CF
:101E7900FEA3E0FFEFD39400EE9408400F900065B5
:101E8900E0B40104C2098002D209800D900065E026
:101E9900B40104D2098002C209900071E07003758F
:101EA9004700900065E07002C20975BB1FE543B4A5
:101EB90003457E017F00E5BE123D22E5BD2FFF509F
:101EC900010E900000EEF0A3EFF07409123D2274A8
:101ED900E68E048F05FF123D048C418D42E54A2DA3
:101EE900FD50010C74018C068D07123D148E418F33
:101EF9004285424A75BB19E543B4040280030220B6
:101F0900787E017F00E5BE123D22E5BD2FFF50011D
:101F19000E900000EEF0A3EFF07404123D148F4B05
:101F2900E564B401028003021FEF756B00756B0055
:101F3900E56BD394074003021FD8E56B900040126C
:101F49003D3AE0D3954B501AE56B900040123D3A6B
:101F5900E0F404254BFEE56B900036123D3AEEF0B5
:101F69008017E56B900040123D3AE0C3954BFEE5C2
:101F79006B900036123D3AEEF0E56BC394044009CC
:101F8900900083E0C3956B503BE56B6029E56B904E
:101F99000036123D3AFEE0FFEE90003EE0D39F404E
:101FA90013E56B900036123D3AE090003EF0E56B88
:101FB90090003FF0800E900036E090003EF07400F3
:101FC90090003FF0786B740126F64003021F3990A8
:101FD900003FE0F4042408F556E556D3940540067D
:101FE900E5B554DFF5B5E564D39401402FE54BD34E
:101FF900946E4004D2158002C215755605E564B485
:102009000205A215B340028003755607E564B403BF
:1020190006A215B3B340028003755607E557655606
:10202900601EE556D39404400DE557D39404400649
:10203900A211B3B340028005D210755A00855657D4
:10204900E556B40708E5B54480F5B58006E5B5540D
:102059007FF5B5E55664066005E556B40808E5B5AB
:102069004410F5B58006E5B554EFF5B575BB13E534
:1020790043B40502800302218C7E017F00E5BE1274
:102089003D22E5BD2FFF50010E900000EEF0A3EFB9
:10209900F07404123D148F46E563B4020280030212
:1020A9002189756B00756B00E56BD39403400302BE
:1020B9002140E56B900032123D3AE0D39546501A23
:1020C900E56B900032123D3AE0F4042546FEE56BDB
:1020D90090002C123D3AEEF08017E56B9000321219
:1020E9003D3AE0C39546FEE56B90002C123D3AEE71
:1020F900F0E56B6029E56B90002C123D3AFEE0FF9C
:10210900EE900030E0D39F4013E56B90002C123D18
:102119003AE0900030F0E56B900031F0800E9000CD
:102129002CE0900030F07400900031F0786B74016D
:1021390026F640030220B1900081E07043E52A456C
:10214900296036E558C39403500A900031E004C36E
:10215900940340028007900031E004F558E558D314
:102169009402400A900031E004D39402500280079F
:10217900900031E004F5588007900031E004F558EB
:1021890075BB180543D2ECA214B3500DAE25AF268A
:1021990074E8C39F74039E4002800575FFA0D214A2
:1021A900AE25AF26EFD39420EE944E50030222A120
:1021B900120321C28E758D00758B00754C00D28E6D
:1021C900C2077571007570007572CD75510575245A
:1021D90000752300755400755A00C2A0900058E09C
:1021E9006004D2978002C297900049E0B40104D2FA
:1021F900958002C295900048E0B40104D29680020D
:10220900C296A209B34004D2A28002C2A290006A77
:10221900E060181233A1A200B34008E5B54408F5FF
:10222900B58006E5B554F7F5B58002C20090006D9A
:10223900E060181234F6A202B34008E5B54402F58D
:10224900B58006E5B554FDF5B58006E5B554FDF54F
:10225900B590000E74FDF0A374E8F0E543B40603ED
:10226900754300C211752600752500758D00758BA3
:1022790000754C00900024E0C3940350089000249A
:10228900E004F080067403900024F0900024E0B488
:102299000306E5B554FEF5B5AE27AF28EFD3941084
:1022A900EE9427401CC2CA75CD0075CC0075280074
:1022B900752700D2CA754E00752A00752900755513
:0422C900000209AC5A
:1036A8000000010001320164019601960200021235
:1036B80002240200020003000340038003C0040048
:1036C8000440048004C00500060006000600060049
:1036D800060006000600060000FF0131016301959F
:1036E80001FF01FF0211022302FF02FF02FF033F55
:1036F800037F03BF03FF043F047F04BF04FF05FFEC
:1037080006FF06FF06FF06FF06FF06FF06FF06FF89
:103718000FAA0FA50F9F0F9A0F940F8D0F870F8079
:103728000F780F710F680F600F570F4E0F450F3B43
:103738000F300F250F1A0F0E0F020EF50EE80EDBD5
:103748000ECC0EBE0EAE0E9F0E8E0E7D0E6C0E5A59
:103758000E470E340E200E0C0DF70DE20DCB0DB5F5
:103768000D9D0D850D6D0D540D3A0D200D050CE9BF
:103778000CCE0CB10C940C760C580C3A0C1B0BFBB1
:103788000BDB0BBB0B9A0B790B570B350B130AF1A1
:103798000ACE0AAB0A870A640A400A1C09F809D447
:1037A80009B0098C09670943091F08FB08D608B244
:1037B800088E086A0846082307FF07DC07B907963A
:1037C80007730751072F070D06EC06CA06AA0689D4
:1037D80006690649062A060A05EC05CD05B00592D4
:1037E80005750558053C0520050504EA04CF04B510
:1037F800049C04820469045104390422040B03F470
:1038080003DE03C803B2039D038903750361034DF7
:10381800033B03280316030402F202E102D102C0AB
:1038280002B002A0029102820273026502570249A5
:10383800023C022F02220216020901FD01F201E6F2
:1038480001DB01D001C601BB01B101A7019D0194B3
:10385800018B0182017901700168016001580150F2
:103868000148014101390132012B0125011E0118CE
:103878000111010B010500FF00FA0FA60FA00F9917
:103888000F920F8B0F840F7C0F740F6B0F620F5802
:103898000F4E0F430F380F2C0F1F0F120F050EF787
:1038A8000EE80ED80EC80EB70EA50E930E800E6C3D
:1038B8000E580E420E2C0E150DFD0DE40DCB0DB15C
:1038C8000D950D790D5D0D3F0D200D010CE10CC01E
:1038D8000C9E0C7C0C590C350C100BEA0BC40B9E7F
:1038E8000B760B4F0B260AFD0AD40AAA0A800A5542
:1038F8000A2A09FF09D409A8097C0950092508F9E9
:1039080008CD08A10875084A081E07F307C8079DCF
:1039180007730749072006F706CE06A6067E065750
:103928000630060A05E405BF059B057705540532F0
:10393800051004EF04CE04AE048F0471045304355B
:10394800041903FD03E203C703AD0394037B036378
:10395800034B0334031E030802F302DE02CA02B655
:1039680002A30291027F026D025C024C023C022C0F
:10397800021D020E020001F201E401D701CA01BED4
:1039880001B101A6019A018F0185017A01700166D2
:10399800015D0153014A0141013901310129012128
:1039A80001190112010B010400FD00F700F000EA03
:1039B80000E400DE00D900D300CE00C900C400BF77
:1039C80000BA00B500B100AD00A800A400A0009C9A
:1039D800009900950091008E008A0087008400817C
:0439E800007E007BE2
:10231B00751A00751900AE19AF1AAC17AD18EDC3CD
:10232B009FEC9E401674FF123CF475CF01781A7423
:10233B000126F6500418E436F650DB22900785E4AC
:10234B00F0A3F0751000750F00751300751400C223
:10235B0016D21722C2AF75D900758F0375B7A57545
:10236B00B7F190F800E4F0758F0175B7A575B7F16B
:10237B00E50890F800F075B7A575B7F190F801E492
:10238B00F075B7A575B7F190079CE090F802F07562
:10239B00B7A575B7F19007A0E090F803F075B7A556
:1023AB0075B7F190079DE090F804F075B7A575B778
:1023BB00F190079EE090F805F075B7A575B7F19011
:1023CB00079FE090F806F075B7A575B7F19007A1D8
:1023DB00E090F807F0758F0075D940D2AF229007C7
:1023EB0087E0B4AB61C2AF75D90075B62275F52223
:1023FB00758F0375B7A575B7F1740090F600F0757E
:10240B008F01750A00750900AE09AF0A7413BE007F
:10241B00279F402475B7A575B7F190078812001E4A
:10242B00E0FC90F60012001EECF0780A740126F620
:10243B00500418E436F650D0758F0075F51175B64B
:10244B002075D940D2AF22C2AF75D90075F5227570
:10245B000A00750900AE09AF0A7413BE00229F4033
:10246B001F90F60012001EE493FC90078812001ECA
:10247B00ECF0780A740126F6500418E436F650D5C1
:10248B0075F51175D940D2AF22900787E0B4AA0237
:10249B0080030225D1C2AF75D90075B62275F5221E
:1024AB00758F0375B7A575B7F1740090EE00F075D5
:1024BB00B7A575B7F1740090F000F075B7A575B7B7
:1024CB00F1740090F200F075B7A575B7F174009038
:1024DB00F400F0758F01750A00750900AE09AF0A9B
:1024EB0074FFC39F74019E402475B7A575B7F19017
:1024FB00004D12001EE0FC90EE0012001EECF07876
:10250B000A740126F6500418E436F650CF750A000B
:10251B00750900AE09AF0A74FFC39F74019E402476
:10252B0075B7A575B7F190024D12001EE0FC90F047
:10253B000012001EECF0780A740126F6500418E421
:10254B0036F650CF750A00750900AE09AF0A74FF55
:10255B00C39F74019E402475B7A575B7F190044DC8
:10256B0012001EE0FC90F20012001EECF0780A74D0
:10257B000126F6500418E436F650CF750A0075099B
:10258B0000AE09AF0A74FFC39F74019E402475B758
:10259B00A575B7F190064D12001EE0FC90F40012E9
:1025AB00001EECF0780A740126F6500418E436F697
:1025BB0050CF758F0075F51175B62075D940D2AF18
:1025CB00743A90074DF022900787E0B4AA0280037B
:1025DB0002270FC2AF75D90075B62275F522758F1C
:1025EB000375B7A575B7F1740090E600F075B7A544
:1025FB0075B7F1740090E800F075B7A575B7F17475
:10260B000090EA00F075B7A575B7F1740090EC0077
:10261B00F0758F01750A00750900AE09AF0A74FFDA
:10262B00C39F74019E402475B7A575B7F190004DFB
:10263B0012001EE0FC90E60012001EECF0780A740B
:10264B000126F6500418E436F650CF750A007509CA
:10265B0000AE09AF0A74FFC39F74019E402475B787
:10266B00A575B7F190024D12001EE0FC90E8001228
:10267B00001EECF0780A740126F6500418E436F6C6
:10268B0050CF750A00750900AE09AF0A74FFC39FDE
:10269B0074019E402475B7A575B7F190044D1200D7
:1026AB001EE0FC90EA0012001EECF0780A74012682
:1026BB00F6500418E436F650CF750A00750900AED3
:1026CB0009AF0A74FFC39F74019E402475B7A575AB
:1026DB00B7F190064D12001EE0FC90EC0012001EAC
:1026EB00ECF0780A740126F6500418E436F650CF55
:1026FB00758F0075F51175B62075D940D2AF743A48
:10270B0090074DF022900787E0B4AA0280030228BD
:10271B004DC2AF75D90075B62275F522758F03754D
:10272B00B7A575B7F1740090DE00F075B7A575B756
:10273B00F1740090E000F075B7A575B7F1740090D7
:10274B00E200F075B7A575B7F1740090E400F07571
:10275B008F01750A00750900AE09AF0A74FFC39F9C
:10276B0074019E402475B7A575B7F190004D12000A
:10277B001EE0FC90DE0012001EECF0780A740126BD
:10278B00F6500418E436F650CF750A00750900AE02
:10279B0009AF0A74FFC39F74019E402475B7A575DA
:1027AB00B7F190024D12001EE0FC90E00012001EEB
:1027BB00ECF0780A740126F6500418E436F650CF84
:1027CB00750A00750900AE09AF0A74FFC39F740147
:1027DB009E402475B7A575B7F190044D12001EE00D
:1027EB00FC90E20012001EECF0780A740126F65001
:1027FB000418E436F650CF750A00750900AE09AF20
:10280B000A74FFC39F74019E402475B7A575B7F179
:10281B0090064D12001EE0FC90E40012001EECF03E
:10282B00780A740126F6500418E436F650CF758FEB
:10283B000075F51175B62075D940D2AF743A900773
:10284B004DF022900787E0B4AA02800302298BC2C5
:10285B00AF75D90075B62275F522758F0375B7A5BF
:10286B0075B7F1740090D600F075B7A575B7F17414
:10287B000090D800F075B7A575B7F1740090DA0029
:10288B00F075B7A575B7F1740090DC00F0758F018A
:10289B00750A00750900AE09AF0A74FFC39F740176
:1028AB009E402475B7A575B7F190004D12001EE040
:1028BB00FC90D60012001EECF0780A740126F6503C
:1028CB000418E436F650CF750A00750900AE09AF4F
:1028DB000A74FFC39F74019E402475B7A575B7F1A9
:1028EB0090024D12001EE0FC90D80012001EECF07E
:1028FB00780A740126F6500418E436F650CF750AA0
:10290B0000750900AE09AF0A74FFC39F74019E40A6
:10291B002475B7A575B7F190044D12001EE0FC901D
:10292B00DA0012001EECF0780A740126F650041837
:10293B00E436F650CF750A00750900AE09AF0A747C
:10294B00FFC39F74019E402475B7A575B7F1900620
:10295B004D12001EE0FC90DC0012001EECF0780A19
:10296B00740126F6500418E436F650CF758F0075B7
:10297B00F51175B62075D940D2AF743A90074DF06A
:10298B0022C2AF75D90075F522750A00750900AE24
:10299B0009AF0A74FFC39F74019E401F90EE001293
:1029AB00001EE493FC90004D12001EECF0780A74AC
:1029BB000126F6500418E436F650D4750A00750952
:1029CB0000AE09AF0A74FFC39F74019E401F90F0C5
:1029DB000012001EE493FC90024D12001EECF078E6
:1029EB000A740126F6500418E436F650D4750A0022
:1029FB00750900AE09AF0A74FFC39F74019E401F97
:102A0B0090F20012001EE493FC90044D12001EEC99
:102A1B00F0780A740126F6500418E436F650D47593
:102A2B000A00750900AE09AF0A74FFC39F74019EBB
:102A3B00401F90F40012001EE493FC90064D120010
:102A4B001EECF0780A740126F6500418E436F650A2
:102A5B00D475F51175D940D2AF22C2AF75D90075B7
:102A6B00F522750A00750900AE09AF0A74FFC39F02
:102A7B0074019E401F90E60012001EE493FC900030
:102A8B004D12001EECF0780A740126F6500418E47F
:102A9B0036F650D4750A00750900AE09AF0A74FFFB
:102AAB00C39F74019E401F90E80012001EE493FC2C
:102ABB0090024D12001EECF0780A740126F65004B9
:102ACB0018E436F650D4750A00750900AE09AF0A42
:102ADB0074FFC39F74019E401F90EA0012001EE416
:102AEB0093FC90044D12001EECF0780A740126F64C
:102AFB00500418E436F650D4750A00750900AE0977
:102B0B00AF0A74FFC39F74019E401F90EC0012002C
:102B1B001EE493FC90064D12001EECF0780A740133
:102B2B0026F6500418E436F650D475F51175D940D5
:102B3B00D2AF22C2AF75D90075F522750A0075099F
:102B4B0000AE09AF0A74FFC39F74019E401F90DE55
:102B5B000012001EE493FC90004D12001EECF07866
:102B6B000A740126F6500418E436F650D4750A00A0
:102B7B00750900AE09AF0A74FFC39F74019E401F15
:102B8B0090E00012001EE493FC90024D12001EEC2C
:102B9B00F0780A740126F6500418E436F650D47512
:102BAB000A00750900AE09AF0A74FFC39F74019E3A
:102BBB00401F90E20012001EE493FC90044D1200A3
:102BCB001EECF0780A740126F6500418E436F65021
:102BDB00D4750A00750900AE09AF0A74FFC39F7460
:102BEB00019E401F90E40012001EE493FC90064DE2
:102BFB0012001EECF0780A740126F6500418E43625
:102C0B00F650D475F51175D940D2AF22C2AF75D934
:102C1B000075F522750A00750900AE09AF0A74FF3D
:102C2B00C39F74019E401F90D60012001EE493FCBC
:102C3B0090004D12001EECF0780A740126F6500439
:102C4B0018E436F650D4750A00750900AE09AF0AC0
:102C5B0074FFC39F74019E401F90D80012001EE4A6
:102C6B0093FC90024D12001EECF0780A740126F6CC
:102C7B00500418E436F650D4750A00750900AE09F5
:102C8B00AF0A74FFC39F74019E401F90DA001200BD
:102C9B001EE493FC90044D12001EECF0780A7401B4
:102CAB0026F6500418E436F650D4750A0075090060
:102CBB00AE09AF0A74FFC39F74019E401F90DC00E6
:102CCB0012001EE493FC90064D12001EECF0780AE5
:102CDB00740126F6500418E436F650D475F51175C8
:102CEB00D940D2AF22E51464046006E59964FF6015
:102CFB00028031A2164004D2168027E514600874B6
:102D0B00E62514900023F0E513600874F02513906A
:102D1B000023F0E514B4010280FE75140075130056
:102D2B00C2168002C216E51490364BF8282873752C
:102D3B001400E599B4FF03751301E599B4FE03750F
:102D4B001302E599B4FD03751303E599B4FC037500
:102D5B001304E599B4FA03751305E599B4FB0675ED
:102D6B001401120321E599B4F90675140412032119
:102D7B00E599D394E54007E599C394F0400280169A
:102D8B008599157514027E017F00E515C394E61233
:102D9B003D228E0D8F0E900785E4F0A3F0E599D3BD
:102DAB0094C44007E599C394E640028028859915A1
:102DBB0075140374E5C39515F50E750D00AE0DAFC7
:102DCB000E9036A812002EE493F8740193900785A9
:102DDB00C8F0A3C8F0D29902325F900785E0FEA33A
:102DEB00E0FFEFC39400EE94054009EFD394FFEEA0
:102DFB0094064013900785E0FEA3E0FF90004D1270
:102E0B00001EE599F0800385996C90078512000EE2
:102E1B00900785E0FEA3E0FFEFB40106EEB40702D6
:102E2B00800302306F90074DE0B43C028003023008
:102E3B006FA20AB35005A20BB34003022F62C29CD0
:102E4B00900079E090078BF0900056E090078CF0A3
:102E5B00900061E090078DF0900062E090078EF09B
:102E6B00900073E090078FF090007BE0900790F05C
:102E7B0090007CE0900791F090007FE0900792F03B
:102E8B00900080E0900793F0900139E0900794F068
:102E9B0090013AE0900795F090013BE0900796F097
:102EAB0090008FE0900797F0900090E0900798F0DB
:102EBB00900091E0900799F0900092E090079AF0C3
:102ECB00900093E090079BF0900094E090079CF0AB
:102EDB00900095E090079DF0900096E090079EF093
:102EEB00900098E090079FF0900099E09007A0F079
:102EFB0090009AE09007A1F090009BE09007A2F061
:102F0B007400900081F012008F74AB900787F01261
:0A2F1B0023E974AA900787F0E55837
:06364B00022D3A022DE5FC
:102F250090366CF82828738012122494800D12258F
:0B2F3500D28008122710800312284EE3
:0F366C00022F2C022F2E022F33022F38022F3D58
:102F4000900787E4F0900139E0700C90013AE0704E
:102F50000690013BE060028004C20A8002D20A02AD
:102F60003064C29C900077E0900788F090005DE0AC
:102F7000900789F090005EE090078AF0900079E079
:102F800090078BF0900056E090078CF0900061E085
:102F900090078DF0900062E090078EF0900073E053
:102FA00090078FF090007BE0900790F090007CE01D
:102FB000900791F090007FE0900792F0900080E001
:102FC000900793F0900139E0900794F090013AE077
:102FD000900795F090013BE0900796F090008FE00D
:102FE000900797F0900090E0900798F0900091E0A3
:102FF000900799F0900092E090079AF0900093E08B
:1030000090079BF0900094E090079CF0900095E072
:1030100090079DF0900096E090079EF0900098E059
:1030200090079FF0900099E09007A0F090009AE040
:103030009007A1F090009BE09007A2F07400900030
:1030400081F074AB900787F01223E974AA90078788
:10305000F01224941225D212271012284ED29C75F9
:1030600099FB80FED29C7514007513007599FB02C4
:10307000325F900785E0FEA3E0FFEF4E7006859972
:1030800010750F00900785E0FEA3E0FF74016F4EFE
:10309000701BAC0FAD10AA0DAB0EED2BFBEC3AFA8A
:1030A0008A068B0790004D12001EE599F090078567
:1030B00012000E900785E0FEA3E0FF74026F4E70D1
:1030C0000C12008F85159975140075130002325F7C
:1030D000900785E0FEA3E0FF90004D12001EE599E9
:1030E000F090078512000E900785E0FEA3E0FFAC8C
:1030F0000DAD0E8F028E038C068D079036E0120008
:103100002EE493F9740193FEEAD39EEB994009856E
:10311000159975140075130002325F900785E0FE63
:10312000A3E0FF90004D12001EE599F09007851274
:10313000000E900785E0FEA3E0FFEFB40006EEB4BA
:103140000102800302325F90001CE0D394C7400B61
:1031500090001CE0C394C8F516801A90001CE0D3C0
:103160009463400B90001CE0C39464F516800690B5
:10317000001CE0F516E51675F002A4FFAEF08F6BAB
:10318000EF90004D123D3AEFFCE0FDEC9000501244
:103190003D3AEDFCE0FDEC2DB51602800302325104
:1031A0000FEF90004D123D3AE56BFFE0FCEF900011
:1031B00051123D3AECFFE0FCEFC39CB516028003D0
:1031C000023251E56B90004F123D3AE56BFFE0FC97
:1031D000EF900052123D3AECFFE0FCEF2CB5167177
:1031E000E56B900053123D3AE0C3951690079CF0B2
:1031F000E56B900054123D3AE0C3951690079DF0A0
:10320000E56B900057123D3AE0C3951690079EF08B
:10321000E56B900058123D3AE0C3951690079FF079
:10322000E56B900059123D3AE0C395169007A0F067
:10323000E56B90005A123D3AE0C395169007A1F055
:1032400012235F7599F975186475170012231B8096
:0F325000FE7599FF75186475170012231B80FE19
:093651000230720230D002311B7C
:10325F0022E51390365AF82828730233A090078579
:10326F00E0FEA3E0FF90001212001EE0F599900718
:10327F008512000E900785E0FEA3E0FF74116F4EDC
:10328F0070037513000233A08562990233A0900773
:10329F0085E0FEA3E0FF90004D12001EE0F599EFD0
:1032AF00B40107EEB4070375130090078512000EE3
:0732BF000233A0900786E036
:0F365A0002326902326C02329702329D0232C292
:1032C60090367BF8282873852499023395852A99A8
:1032D600023395854499023395854799023395853E
:1032E6005199023395856099023395855699023333
:1032F60095855899023395756E00900068E07006C2
:10330600900067E060028016A2A44006E56E4404C1
:10331600F56EA2A54006E56E4402F56E801A900091
:1033260049E0B40106E56E4410F56E900048E0B43D
:103336000106E56E4420F56EA207B34006E56E442D
:1033460001F56EA209B34006E56E4408F56E856E7A
:1033560099803CA217B340077599FAC2178017A245
:103366000CB3400575990F800B900023E0F59990FA
:103376000023E4F0C20C80178542998012854B9990
:0F338600800D85469980087599FC8003751300AA
:10367B000232CD0232D30232D90232DF0232E502FC
:10368B0032EB0232F10232F70232FD0233590233CE
:0D369B007E02338302338802338D023392A6
:0B33950090078512000E800312004814
:0336690002339D8C
:1033A0002290006AE0B4010385241190006AE0B421
:1033B0000203852A1190006AE0B40303854411904A
:1033C000006AE0B4040385471190006AE0B4050385
:1033D00085511190006AE0B4060385561190006A89
:1033E000E0B4070385581190006BE0FE90006CE09C
:1033F000C39E500302347790006AE0D39404402CBB
:1034000090006BE0D39511500990006CE0C39511CA
:1034100050028002D20090006BE0D39511500990C9
:10342000006CE0C395115002C200804990006AE030
:10343000B4041890006CE0C395115002D2009000C3
:103440006BE0D395114002C200802A90006BE0C36C
:103450009511500990006CE0D3951150028002D272
:103460000090006BE0D39511500990006CE0C3957B
:10347000115002C200807E90006AE0D39404402C78
:1034800090006BE0C39511400990006CE0D395115A
:1034900040028002C20090006BE0C3951140099089
:1034A000006CE0D395114002D200804990006AE0A0
:1034B000B4041890006BE0C395115002C200900054
:1034C0006CE0D395114002D200802A90006BE0C3DB
:1034D0009511400990006CE0D395114002D2009004
:1034E000006BE0D39511400990006CE0C39511404A
:1034F000028002C2002290006DE0B4010385241115
:1035000090006DE0B40203852A1190006DE0B403D1
:103510000385441190006DE0B404038547119000C9
:103520006DE0B4050385511190006DE0B40603858C
:10353000561190006DE0B4070385581190006EE0BD
:10354000FE90006FE0C39E50030235CC90006DE00A
:10355000D39404402C90006EE0D395115009900054
:103560006FE0C3951150028002D20290006EE0D34A
:103570009511500990006FE0C395115002C202806E
:103580004990006DE0B4041890006FE0C3951150AD
:1035900002D20290006EE0D395114002C202802A4E
:1035A00090006EE0C39511500990006FE0D3951123
:1035B00050028002D20290006EE0D3951150099023
:1035C000006FE0C395115002C202807E90006DE052
:1035D000D39404402C90006EE0C3951140099000F4
:1035E0006FE0D3951140028002C20290006EE0C3EA
:1035F0009511400990006FE0D395114002D20280EE
:103600004990006DE0B4041890006EE0C39511502D
:1036100002C20290006FE0D395114002D202802ACC
:1036200090006EE0C39511400990006FE0D39511B2
:103630004002D20290006EE0D39511400990006FD5
:0B364000E0C3951140028002C202228C
:093D3A002582F582500205832266
:10002E00EF2F500205832582F582E5833E2EF58360
:01003E00229F
:08000300C3EF9DFFEE9CFE22FD
:08003F000806B60002180622B3
:0D000E00A3E004F07006123D30E004F02283
:083D4C000816B6FF021816224A
:0E3D1400048007C3CE13CECF13CFD5E0F62226
:103BC200BC000FBE0008ED8FF084FFADF022E4FED2
:103BD200FF22BE000DEF60FE54F0606F20E703028B
:103BE2003C78EAC0E0EBC0E078017A0075F001EEC3
:103BF20020E710EF25E0FFEE33FE0AC5F023C5F003
:103C020030E7F0EA5407F9096A7A007B006001089C
:103C1200C3EC9E40167004ED9F4010ED9FFDEC9E9C
:103C2200FCE5F0CA4ACA03F5F08005E5F003F5F0B9
:103C3200C3EE13FEEF13FFD9D77908CACBCAD8D087
:103C4200EAFEEBFFD0E0FBD0E0FA22EC8FF084FC3E
:103C5200ED54F045F0C48FF084FEEDC454F045F00D
:103C6200C48FF084FDEEC4FE54F02DFFEE540F3CE1
:103C7200FEADF07C0022790078008FF0EC7E082007
:103C8200E70DC3CD33CD33C933C9C833C8DEF084A1
:103C920049F9E5F08FF0BE00E6FD7C00E9FFE8FEA1
:013CA20022FF
:0E3D2200F88FF0A4FFE5F0CE88F0A42EFE226C
:103CF400600D782B023CFE007830D8FED5E0F82227
:103D0400EEC0E07E00123BC2EFFDEEFCD0E0FE22EE
:03000B00023CA311
:03001B00023CBEE6
:03002B00023CD9BB
:03000000023D437B
:093D430075817375D00002050BB7
:0B001E00E5822FF582E5833EF583228A
:0A3D30000582D58202158315822258
:103CA300C0E0C0F0C083C082C0D075D00012050050
:103CB300D0D0D082D083D0F0D0E032C0E0C0F0C00A
:103CC30083C082C0D075D000120503D0D0D082D07B
:103CD30083D0F0D0E032C0E0C0F0C083C082C0D057
:103CE30075D000120506D0D0D082D083D0F0D0E0BA
:013CF300329E
:00000001FF
